:020000040000FA
:10000000FDEF00F0F76A140FF66E000EF7220900FC
:10001000F55012000A0A0D2A2A2A2A2A2A2A2A2AEE
:100020002A2A2A2A2A2A2A2A20303235202D205705
:100030006972656C657373204D756C74694D657478
:100040006572205458202A2A2A2A2A2A2A2A2A2A49
:100050002A2A2A2A2A2A2A2A2A200A0A0D00F76A84
:100060006E0FF66E000EF7220900F5501200696E51
:100070006974204F4B200A0D00001FBE10D00F0ED8
:10008000006E1E3800160A0E005C03E2300E0026D9
:1000900002D01F50002600509EA8FED7AD6E0F0E56
:1000A0001E160A0E1E5C02E2300E02D01F9E1F506A
:1000B0001E261E509EA8FED7AD6E000C296A295040
:1000C00018080EE3828A290E006E002EFED700006B
:1000D000829A290E006E002EFED70000292AEFD743
:1000E000828A7C0E006E002EFED700000000829AED
:1000F0007C0E006E002EFED700000000828A7C0E6F
:10010000006E002EFED700000000829A7C0E006E6A
:10011000002EFED700000000DCEF00F0828AA60E61
:10012000006E002EFED70000829A290E006E002E6F
:10013000FED70000E3EF00F0828A290E006E002E49
:10014000FED7000008A005D0290E006E002EFED7B5
:100150000000829A290E006E002EFED70000BFEF2D
:1001600000F007C029F0080E066E06520FE0295075
:10017000800B800802E1088001D00890DDD706508E
:10018000010802E2D89029360606EFD7EDEF00F01D
:10019000AA0E1E6EA50E1F6E0AC020F00BC021F025
:1001A0000CC022F00DC023F009C024F0256ACC0E4B
:1001B000266EAA0E276E82D7056A05BE03D00550AB
:1001C00009080DE3ABD7036A05501E0FE96E000E58
:1001D0000320EA6EEFCF07F0C4D7052AEED7828A54
:1001E000290E006E002EFED70000829A290E006EA6
:1001F000002EFED7000069EF02F0F86AD09EFE0ED6
:10020000006E060E016E020EE96E000EEA6EEF6AD7
:10021000E92AD8B4EA2A002EFAD7012EF8D7EA6ADA
:10022000E96A0C0EAF6E260EAC6E900EAB6EC180FE
:10023000C182C184C196FE0E926EFF0E936E9F0E18
:10024000946EFF0E956E9680968296848080C29002
:100250001E6A1E50D7DE000905E01E2A9EA8FED7A2
:10026000AD6EF7D71E6A1E50FADE000905E01E2AA1
:100270009EA8FED7AD6EF7D7809082A801D0FDD79B
:10028000000000000000000083501F0B096E80CFAB
:100290000EF081CF0FF082CF10F083CF11F084CF1A
:1002A00012F00892089408960898089A136A146A3B
:1002B000156A0A6A0B6A0C6A0D6A11AA02D0010E4D
:1002C0000A6E10B6138C11BE138A11BC13880EB8B7
:1002D000138610B213840EBA138210B41380135015
:1002E000060803E1010E0B6E39D013505B0803E1E1
:1002F000020E0B6E33D013504F0803E1030E0B6E4A
:100300002DD01350660803E1040E0B6E27D0135056
:100310006D0803E1050E0B6E21D013507D0803E13B
:10032000060E0B6E1BD01350070803E1070E0B6E71
:1003300015D013507F0803E1080E0B6E0FD0135039
:100340006F0803E1090E0B6E09D013503F0802E15C
:100350000B6A04D0135202E10F0E0B6E10B0148C16
:100360000EB4148A0EB614880FB814860FBA14840B
:100370000FBC14820FBE14801450060803E1010E56
:100380000C6E39D014505B0803E1020E0C6E33D0B2
:1003900014504F0803E1030E0C6E2DD01450660864
:1003A00003E1040E0C6E27D014506D0803E1050E16
:1003B0000C6E21D014507D0803E1060E0C6E1BD08C
:1003C0001450070803E1070E0C6E15D014507F0877
:1003D00003E1080E0C6E0FD014506F0803E1090EF4
:1003E0000C6E09D014503F0802E10C6A04D014527C
:1003F00002E10F0E0C6E0FB4158C0FB2158A0FB6FA
:10040000158812B4158612B2158412B015820FB079
:1004100015801550060803E1010E0D6E39D01550F8
:100420005B0803E1020E0D6E33D015504F0803E157
:10043000030E0D6E2DD01550660803E1040E0D6EEF
:1004400027D015506D0803E1050E0D6E21D0155013
:100450007D0803E1060E0D6E1BD01550070803E161
:10046000070E0D6E15D015507F0803E1080E0D6EB6
:100470000FD015506F0803E1090E0D6E09D015500D
:100480003F0802E10D6A04D0155202E10F0E0D6E15
:100490000AC01EF0D70E1F6EF0DD0BC01EF0D70E87
:1004A0001F6EEBDD0CC01EF0D70E1F6EE6DD0DC01B
:1004B0001EF0D70E1F6EE1DD200E9EA8FED7AD6E9A
:1004C0000A0E9EA8FED7AD6E0D0E9EA8FED7AD6E8D
:0604D0005FD6D3D6030045
:00000001FF
